:020000040800F2
:1000000000040020E1010008E3010008E30100080A
:10001000E3010008E3010008E3010008E301000830
:10002000E3010008E3010008E301000825250008BA
:10003000E3010008E3010008E3010008E301000810
:10004000E3010008E3010008E3010008E301000800
:10005000E3010008E301000885360008B136000816
:10006000DD3600080937000835370008E3010008CD
:10007000E3010008E3010008E3010008E3010008D0
:10008000E3010008E3010008E3010008E3010008C0
:10009000E3010008E3010008E301000861370008FC
:1000A000E3010008E3010008E3010008E3010008A0
:1000B000E3010008E3010008E3010008E301000890
:1000C000E3010008E3010008E3010008E301000880
:1000D000E3010008E3010008910E0008E3010008B5
:1000E000C9370008E3010008E3010008E301000844
:1000F000E3010008E3010008E3010008E301000850
:10010000E3010008E30100089D340008E301000852
:10011000E3010008E3010008E3010008E30100082F
:10012000E3010008E3010008E3010008E30100081F
:10013000E3010008E3010008E3010008E30100080F
:10014000E3010008E3010008E3010008112C0008A6
:10015000E3010008E3010008E3010008E3010008EF
:10016000E3010008E3010008E3010008E3010008DF
:10017000E3010008E3010008E3010008E3010008CF
:10018000E3010008E3010008E3010008E3010008BF
:10019000E3010008E3010008E3010008E3010008AF
:1001A000E3010008E3010008E3010008E30100089F
:1001B000E3010008E3010008E3010008E30100088F
:1001C000E3010008E3010008E3010008E30100087F
:1001D000E3010008E3010008E3010008E30100086F
:1001E00002E000F000F8FEE772B6394880F30888B4
:1001F000384880F3098838484EF60851CEF200019D
:10020000086040F20000CCF200004EF63471CEF2ED
:1002100000010860BFF34F8FBFF36F8F40F2000003
:10022000C0F2F0004EF68851CEF200010860BFF334
:100230004F8FBFF36F8F4FF00000E1EE100A4EF6C4
:100240003C71CEF200010860062080F31488BFF3F1
:100250006F8F02F0A5F903F0B7F84FF055301F4942
:100260001B4A91423CBF41F8040BFAE71C49194A6A
:1002700091423CBF41F8040BFAE71A491A4A1B4B5A
:100280009A423EBF51F8040B42F8040BF8E70020F5
:100290001749184A91423CBF41F8040BFAE702F0B3
:1002A00083F903F0EDF8144C144DAC4203DA54F822
:1002B000041B8847F9E700F03FF8114C114DAC42A0
:1002C00003DA54F8041B8847F9E702F06BB9000021
:1002D000000400200024002000000008000000208E
:1002E00000040020383C00080024002028240020BE
:1002F0002824002090380020E0010008E0010008D8
:10030000E0010008E00100082DE9F04F2DED108A12
:10031000C1F80CD0C3689D46BDEC108ABDE8F08FD3
:10032000002383F311882846A047002001F0C4FD74
:1003300001F074FD00DFFEE71B4B142270B51A704C
:100340006FF03F0200245A720F225C709C70DC70C8
:100350001C715C719C71DC711C729A72DC7202F00F
:10036000AFF8064602F0D8F8054650B90F4B9E424A
:1003700017D001339E4241F2883412BF0546002453
:100380000125002002F0A2F80DB100F0B5F800F050
:1003900011FD00F0E5FB204600F00CF900F0ACF890
:1003A000F9E70446EDE700BF28240020010007B06C
:1003B00008B500F053FBA0F120035842584108BD96
:1003C00007B5054B02211B88ADF8043001A800F0E9
:1003D000B1FB03B05DF804FBC8380008064991F88A
:1003E000243033B100230822086A81F8243000F059
:1003F000D9BB0120704700BF482400202DE9F84FE9
:10040000234C94F824300546884617468BBB2E466D
:10041000DFF87C90002F38D094F824A0BAF1000FB8
:1004200005D12022FF214846266200F0B1FCCAF126
:100430000805BD4228BF3D465FFA85FBAD00414639
:100440002A4604EB8A0000F079FC94F82430A7EBEC
:100450000B079B445FFA8BFBBBF1080F2E44A844AB
:10046000FFB284F824B0D5D1FFF7B8FF0028D1D16E
:1004700008E0266A06EB8306B042C9D0FFF7AEFF5C
:100480000028C4D10020BDE8F88F0120BDE8F88F16
:100490004824002010B5202383F311881248C36834
:1004A0000BB101F08FFD0023104A0F484FF47A7111
:1004B00001F04CFD002383F311880D4C236813B128
:1004C0002368013B2360636813B16368013B636089
:1004D000084B1B7833B9636823B9022000F01CFC79
:1004E0003223636010BD00BF34240020950400084F
:1004F000782900207024002010B5254B254953F899
:10050000042F013200D110BD8B42F8D1224C234B75
:1005100022689A423AD9224B9B6803F1006303F5A3
:1005200080439A4232D2002000F034FB1D4B02205F
:10053000187000F0E3FB1C4B1A6C00221A64196E51
:100540001A66196E596C5A64596E5A665A6E5A690F
:1005500042F080025A615A6922F080025A615A6957
:100560001A6942F000521A611A6922F000521A61A7
:100570001B6972B60D4A0E4B13601B68226820215E
:1005800081F311889D4683F30888104710BD00BF92
:10059000FC3F00081C40000804400008FF3F000822
:1005A00028240020702400200038024008ED00E0DC
:1005B000004000082DE9F04FB54C97B0202282464C
:1005C000FF210EA8A56800F0E3FBB24A1378A0460D
:1005D000A3B9B1480121C3601170202383F31188AE
:1005E000C3680BB101F0EEFC0023AC4AAA484FF4FB
:1005F0007A7101F0ABFC002383F31188DFF8BCB201
:10060000BAF1000F01D0CBF800A0A54F00243C7038
:10061000CBF804402646012000F070FBBAF1000F31
:1006200000F0E081DBF80030002B40F0DB8117B0F8
:10063000BDE8F08F0220FFF7BBFE002840F0D0811C
:10064000984B1B88ADF82430022109A800F072FAFB
:10065000E1E74FF47A7000F001FA031E0193EFDB3B
:100660000220FFF7A5FE81460028E9D0019B581E15
:100670000428E5D8DFE800F0030C0F12150016A8D7
:10068000052340F8343D042100F054FA4C4650E074
:1006900004217F48F8E704218348F5E704218348D3
:1006A000F2E71C24204600F077FA04340990042174
:1006B00009A800F03FFA2C2CF4D1E7E7002EBFD0B8
:1006C000002CBDD00220FFF773FE064610B90124AE
:1006D0002646B5E7012000F05DFA0220387000F0F0
:1006E0000DFB0024E3B21846019300F063FA814643
:1006F00048B1019B184600F06DFA01340028F1D191
:1007000034466B4B9DE7012302203B7000F0EAFA70
:100710004D46D8F808309D4206D2284600F03CFAF3
:100720000130EDD10435F4E700253D70CBF80450DD
:10073000344600F035FBFFF743FE4EE1002E3FF458
:100740007FAF002C3FF47CAF0220387000F0D6FA67
:10075000322000F083F9041EB9DB14F00306B6D191
:10076000D8F808202B199342B1D8B4F5807FAED8C1
:10077000DFF84091A6420CDA4FF47A7000F06EF97F
:100780000390039B002BA2DB039B06F80930013684
:10079000F0E7C820FFF70CFE0646002897D01F2D73
:1007A00011D8C5F12009A14528BFA1460EAB25F0FF
:1007B00003004A463F49184400F0C0FA4A46FF2168
:1007C0003C4800F0E5FA4FEAA4095FFA89F239499A
:1007D0002846FFF713FE0446002891D005EB890553
:1007E0000646A6E70220FFF7E3FD00283FF428AF06
:1007F000FFF7F4FD00283FF423AF4FF0000AD14685
:10080000D8F808309A453CD2BAF11F0F1CD80E9B7D
:10081000013319D02AF0030316AA134453F8203CDD
:10082000099325494B68A3B1002209A8135C83EA08
:100830000903DBB2013251F82330042A83EA192973
:10084000F4D10AF1040ADBE7504600F0A5F909905B
:10085000E7E71A46082012F0010F4FEA52021FBFC5
:1008600082F06D4282F4380282F4034282F0200268
:100870000138F0D141F823200133B3F5807FE8D16E
:10088000D2E716A8042140F8489D00F053F950E73C
:10089000282400207425002034240020950400081A
:1008A00070240020CA3800082C24002030240020A6
:1008B000CC380008742400207825002078290020F6
:1008C00016A8002340F8343D642100F0FFF800280A
:1008D0007FF4B6AE0220FFF76BFD00283FF4B0AE08
:1008E000099800F089F916AB43F8440D0421184625
:1008F000CBE716A8002340F8343D642100F0E6F869
:1009000000287FF49DAE0220FFF752FD00283FF43F
:1009100097AE099800F07EF916AB43F8400DE5E775
:100920000220FFF745FD00283FF48AAE00F078F979
:1009300016AB43F83C0DD9E70220FFF739FD00283C
:100940003FF47EAE09A9142000F070F9814616A884
:10095000042140F8389D00F0EDF8494609A894E7D5
:100960004FF47A70FFF724FD00283FF469AEFFF7DB
:1009700035FD00283FF4C5AE0E9B01330CD0082294
:100980000EA90020FFF73AFD00283FF4BAAE20225E
:10099000FF210EA800F0FCF9FFF712FD2E4801F030
:1009A00091FA44E616A8002340F8343D642100F093
:1009B0008DF800287FF444AE0220FFF7F9FC0028F0
:1009C0003FF43EAEFFF7FCFC41F2883001F07AFACA
:1009D000099800F029FA00F0E3F94FF0000A1AE64E
:1009E0000646A6E6002000F039F80390039B002B92
:1009F000FFF614AE012000F075F9039B213B122B8A
:100A00003FF609AE01A252F823F000BF35060008F8
:100A100053060008BD060008170600081706000860
:100A2000170600083D07000817060008E50700083C
:100A3000C1080008F308000821090008170600088B
:100A40003909000817060008610900083307000883
:100A500017060008A5090008A08601002DE9F34744
:100A600002AE00244FF47A7506F8014D144FDFF8FA
:100A70005880454397F900305A1C5FFA84F901D039
:100A8000A34212D158F8240003680122D3F820A011
:100A900031462B46D047012807D10A4B9DF8070065
:100AA00083F8009002B0BDE8F0870134022CE1D158
:100AB0004FF4FA7001F006FA4FF0FF30F2E700BF92
:100AC00000240020982900200C3900082DE9F04767
:100AD0004FF47A75144FDFF8588006464D430024D2
:100AE00097F900305A1C5FFA84F901D0A34210D163
:100AF00058F8240003680422D3F820A031462B467E
:100B0000D047042805D1094B83F800900020BDE8A8
:100B1000F0870134022CE3D14FF4FA7001F0D2F9DE
:100B20004FF0FF30BDE8F087002400209829002016
:100B30000C39000830B4074B1A78074B53F82240A1
:100B40002368DD69054B0A46AC460146204630BCA9
:100B5000604700BF982900200C390008A0860100DA
:100B600070B501F0EFFB094C094E2070002530688C
:100B70002378834208D901F0DFFB33680544013351
:100B8000B5F5804F3360F2D370BD00BF99290020C6
:100B90008029002001F080BC00F1006000F5804059
:100BA0000068704700F10060920000F5804001F09D
:100BB0000BBC0000054B1A68054B1B789B1A83423F
:100BC00002D9104401F0B8BB0020704780290020F2
:100BD0009929002038B5074D04462868204401F0C3
:100BE000B3FB28B928682044BDE8384001F0C4BBF5
:100BF00038BD00BF8029002010F0030308D1B0F5F4
:100C0000007F05D800F10050A0F50840006870474B
:100C100000207047014BC058704700BF107AFF1F7B
:100C2000014B1868704700BF002004E070B52A4BE4
:100C30001C68C4F30B03240C63B140F213429342CB
:100C400031D040F2194293422FD040F221429342D8
:100C50002DD10323214A0C2505FB03235D6893F95D
:100C6000082042F201039C4224D0B4F5805F23D0D7
:100C700041F201039C4221D041F203039C421FD068
:100C800041F207039C4208BF3122441E0C44013D3F
:100C90000B46A3421ED215F9016F581C96B10346AC
:100CA00000F8016CF5E70123D4E70223D2E73F22E5
:100CB0000B4DD6E73322E3E74122E1E75A22E4E78E
:100CC0005922E2E72C2584421D7001D9981C5A70E4
:100CD000401A70BD1846FBE7002004E0DC3800082D
:100CE000D0380008022803D10822034B9A617047CC
:100CF0000128FCD10422F8E700100240022804D1A8
:100D00004FF40022034B9A6170470128FCD14FF445
:100D10008022F7E700100240022805D1064A5369F5
:100D200083F00803536170470128FCD1024A5369DC
:100D300083F00403F6E700BF0010024010B5002363
:100D4000934203D0CC5CC4540133F9E710BD0000DA
:100D500030B5441E14F9010F0B4660B193F90050F1
:100D6000854201F1010106D11AB993F90020801AD8
:100D700030BD013AEEE7002AF7D1104630BD000041
:100D800002460346981A13F9011B0029FAD170474D
:100D900002440346934202D003F8011BFAE770476E
:100DA000024B1A78024B1A70704700BF9829002036
:100DB0000024002038B5164D164C284600F0CAFB1A
:100DC0002146284600F0F2FB236813485A6DD2F8FA
:100DD000043843F00203C2F8043801F073F80F49F5
:100DE000206800F0EFFC23680D485A6D0D49D2F8D9
:100DF000043823F00203C2F80438A8424FF4E13368
:100E00000B6003D0BDE8384000F002BB38BD00BF26
:100E1000442E0020EC39000840420F00343A00080C
:100E20009C2900208429002038B50B4B1A780B4BE5
:100E300053F822400A4B9C4205460CD0094B002136
:100E400018461422FFF7A4FF056001462046BDE8BE
:100E5000384000F0DDBA38BD982900200C39000870
:100E6000442E002084290020024AD36843F0C003A6
:100E7000D360704700440040044B5A6810439A689E
:100E800058600AB1181D1047704700BF9C29002008
:100E90002DE9F0413D4ED6F85C54EF682B68DA0539
:100EA0009CB20CD5202383F311884FF40070FFF718
:100EB000E3FF6FF480732B60002383F311882023FA
:100EC00083F31188DFF8C48014F02F0331D183F34A
:100ED0001188380613D5210611D5202383F31188F4
:100EE0002B4800F0F3F9002844DA0820FFF7C4FF8C
:100EF0004FF67F733B40EB60002383F311887A0643
:100F00000DD563060BD5202383F31188F26C336D66
:100F10009A4201D1336C7BBB002383F31188D6F84E
:100F20006424D3680BB110699847BDE8F04101F023
:100F300009BB230712D014F0080F0CBF002080203B
:100F4000E10748BF40F02000A20748BF40F0400042
:100F5000630748BF40F48070FFF78EFFA4066B68FC
:100F600005D596F860144046194000F05FFA2C68E9
:100F7000A4B2A9E76860BFE727F040073F0410204C
:100F80003F0CFFF779FFEF60C6E700BF9C29002008
:100F9000D429002010B5054C054A0021204600F058
:100FA00015FA044BC4F85C3410BD00BF9C29002026
:100FB000690E00080044004038B5294C037C002924
:100FC00018BF0C46012B0546C0F8644410D1254BD0
:100FD00098420DD1244B1A6C42F400321A641A6EF6
:100FE00042F400321A660B2126201B6E00F046F8F0
:100FF0001E4BD5F85C249A42236802D01C498A42D1
:101000002BD11C4901EB5301B1FBF3F3A188080478
:1010100042BF23F0070003F0070343EA4003936055
:10102000E38843F040039BB21361238943F001033B
:101030009BB2536141F4045343F02C03D36001F499
:10104000A05100231360B1F5806F136853680CBF83
:101050007F23FF2385F8603438BD0749D2E700BFFE
:10106000343900089C29002000380240001001405B
:101070000014014000BD010580DE800200F16043E4
:1010800000F01F02400903F5614309018000C9B265
:1010900000F1604083F8001300F5614001239340A4
:1010A000C0F8803103607047F8B51546826806695C
:1010B000AA420B46816938BF8568761AB542044654
:1010C00007D218462A46FFF739FEA3692B44A361CD
:1010D0000DE011D932461846FFF730FEAF1B3A46F5
:1010E000E1683044FFF72AFEE2683A44A261A3684F
:1010F0005B1BA3602846F8BD18462A46FFF71EFE74
:10110000E368E4E783682DE9F0410446934215461D
:10111000266938BF85684069361AB5420F4606D23F
:101120002A46FFF70BFE63692B4463610DE012D979
:101130003246A5EB0608FFF701FE4246B919E06802
:10114000FFF7FCFDE26842446261A3685B1BA36099
:101150002846BDE8F0812A46FFF7F0FDE368E4E7A2
:1011600010B50A440024C361029B006040608460A3
:10117000C160816141610261036210BD08B582698D
:101180004369934201D1826882B9826801328260E8
:101190005A1C42611970426903699A4201D3C368BB
:1011A0004361002100F0AAFE002008BD4FF0FF308F
:1011B00008BD000070B5202304460E4683F3118855
:1011C000A568A5B1A368A269013BA360531CA361F4
:1011D00015782269934224BFE368A361E3690BB1E8
:1011E00020469847002383F31188284670BD314676
:1011F000204600F073FE0028E2DA85F3118870BD06
:101200002DE9F74F05460F4690469A46D0F81C90B8
:10121000202686F311884FF0000B144664B1224655
:1012200039462846FFF740FF034668B9514628462D
:1012300000F054FE0028F1D0002383F31188A8EBBE
:10124000040003B0BDE8F08FB9F1000F03D00190A6
:101250002846C847019B8BF31188E41A1F4486F384
:101260001188DBE7C16081614161C3611144009B6A
:10127000006040608260016103627047F8B5044617
:101280000E461746202383F31188A568A5B1A368ED
:10129000013BA36063695A1C62611E702369626925
:1012A0009A4224BFE3686361E3690BB12046984723
:1012B000002080F31188F8BD3946204600F00EFE6C
:1012C0000028E2DA85F31188F8BD000083694269DD
:1012D0009A4210B501D182687AB98268013282607F
:1012E0005A1C82611C7803699A4201D3C3688361E6
:1012F000002100F003FE204610BD4FF0FF3010BD6E
:101300002DE9F74F05460F4690469A46D0F81C90B7
:10131000202686F311884FF0000B144664B1224654
:1013200039462846FFF7EEFE034668B9514628467F
:1013300000F0D4FD0028F1D0002383F31188A8EB3E
:10134000040003B0BDE8F08FB9F1000F03D00190A5
:101350002846C847019B8BF31188E41A1F4486F383
:101360001188DBE7026843681143016003B1184745
:10137000704700001430FFF743BF00004FF0FF3309
:101380001430FFF73DBF00003830FFF7B9BF000051
:101390004FF0FF333830FFF7B3BF00001430FFF7D2
:1013A00009BF00004FF0FF311430FFF703BF00000A
:1013B0003830FFF763BF00004FF0FF323830FFF7DF
:1013C0005DBF000000207047FFF7E4BD37B50F4B4D
:1013D0000360002343608360C360012304460374F9
:1013E000154600900B464FF4007200F15C0114307A
:1013F000FFF7B6FE00942B464FF4007204F5177108
:1014000004F13800FFF72EFF03B030BD4839000863
:1014100010B52023044683F31188FFF7CDFD022386
:101420002374002383F3118810BD000038B5C3690D
:1014300004460D461BB904210844FFF793FF2946D3
:1014400004F11400FFF79AFE002806DA201D4FF47D
:101450008061BDE83840FFF785BF38BD026843684A
:101460001143016003B118477047000013B5446B86
:10147000D4F894341A681178042915D1217C0229F2
:1014800012D11979128901238B4013420CD101A981
:1014900004F14C0001F00CFED4F89444019B217936
:1014A0000246206800F0DAF902B010BD143001F0F5
:1014B0008FBD00004FF0FF33143001F089BD0000F4
:1014C0004C3001F061BE00004FF0FF334C3001F0B2
:1014D0005BBE0000143001F05DBD00004FF0FF3135
:1014E000143001F057BD00004C3001F02DBE00005B
:1014F0004FF0FF324C3001F027BE0000D0F89424AA
:1015000038B5136819780429054601D0012038BD83
:10151000017C0229FAD112795C89012090400440B3
:10152000F4D105F1140001F0EFFC02460028EDD0E3
:10153000D5F894544FF480732868697900F07CF9E9
:10154000204638BD406BFFF7D9BF00000020704730
:10155000704700007FB5124B036000234360836037
:10156000C360012502260F4B0574044602900193C7
:1015700000F18402294600964FF48073143001F084
:101580009FFC094B0193029400964FF4807304F57D
:101590002372294604F14C0001F066FD04B070BDD1
:1015A00070390008451500086D1400080B682022EA
:1015B00082F311880A7903EB820290614A79093239
:1015C00043F822008A7912B103EB82039861022367
:1015D0000374C0F89414002383F31188704700004B
:1015E00038B5037F044613B190F85430ABB9201DD1
:1015F00001250221FFF732FF04F1140025776FF077
:10160000010100F087FC84F8545004F14C006FF0A5
:101610000101BDE8384000F07DBC38BD10B50121A6
:1016200004460430FFF71AFF0023237784F8543070
:1016300010BD000038B504460025143001F058FCF8
:1016400004F14C00257701F027FD201D84F854504B
:101650000121FFF703FF2046BDE83840FFF74EBFEA
:1016600090F8443003F06003202B19D190F8452006
:10167000212A0AD0222A4FF000030ED0202A0FD1AF
:10168000084A82630722C26304E0064B8363072390
:10169000C36300230364012070478363C363F9E7D6
:1016A0000020704701240020D0F8943437B51A6820
:1016B0001178042904461AD1017C022917D119791D
:1016C000128901238B40134211D100F14C052846A9
:1016D00001F0A2FD58B101A9284601F0E9FCD4F8B7
:1016E0009444019B21790246206800F0B7F803B0CA
:1016F00030BD000000EB8103F7B59C6905460E463E
:10170000F4B1202383F3118805EB8607201D0821FF
:10171000FFF7A4FEFB685B691B684C3413B12046DD
:1017200001F0D4FC01A9204601F0C2FC024648B1F8
:10173000019B3146284600F091F8002383F311887D
:1017400003B0F0BDFB685A691268002AF5D01B8A05
:10175000013B1340F1D105F14402EAE7093138B504
:1017600050F82140DCB1202383F31188D4F894246D
:101770001368527903EB8203DB689B695D6845B1AE
:1017800004216018FFF76AFE294604F1140001F0F5
:10179000C5FB2046FFF7B2FE002383F3118838BD56
:1017A0007047000000F086BF0123037000234360F0
:1017B000C36183620362C362436203630381438143
:1017C0007047000038B50446202383F311880025B4
:1017D0004160C56005614561856100F07BFF0223C2
:1017E000237085F3118838BD70B500EB8103054681
:1017F0005069DA600E46144618B110220021FFF736
:10180000C7FAA06918B110220021FFF7C1FA3146CA
:101810002846BDE8704001F027B80000028902F0B8
:1018200001020281428902F001024281002202612A
:101830004261826101F0ACB8F0B400EB81044789E9
:10184000E4680125A4698D403D4345812360002360
:10185000A2606360F0BC01F0C7B80000F0B400EB18
:1018600081040789E468012564698D403D43058151
:1018700023600023A2606360F0BC01F041B9000066
:1018800070B50223002504460370A0F84C5080F880
:101890004E5080F84F5005814581C5600561456116
:1018A000856180F8345000F07BFF63681B6823B1CA
:1018B00029462046BDE87040184770BD436802784D
:1018C0001B6880F85020052202700BB104211847D4
:1018D00070470000436890F850201B6802700BB1FD
:1018E000052118477047000090F8343070B5044661
:1018F00013B1002380F8343004F14402204601F093
:1019000069F863689B6863BB94F8445015F06006FF
:1019100015D194F8453005F07F0545EA032540F2DE
:1019200002339D4200F00E815BD8022D00F0DC8076
:101930003FD8002D00F08780012D00F0CF800021DE
:10194000204601F09FFA0021204601F091FA6368D9
:101950001B6813B1062120469847062384F83430CB
:1019600070BD204698470028CED094F84B2094F8BC
:101970004A3043EA0223E26B934238BFE36394F9AF
:101980004430E56B002B4FF0200380F2FD80002DEA
:1019900000F0EC80092284F8342083F311880021C0
:1019A000E36BA26B2046FFF759FF002383F31188F6
:1019B00070BDB5F5817F00F0B180B5F5407F49D0AD
:1019C000B5F5807FBBD194F84630012BB7D1B4F880
:1019D0004C3023F00203A4F84C30A663E66326647F
:1019E000C3E740F201639D421ED8B5F5C06F3BD2FC
:1019F000B5F5A06FA3D1B4F84430B3F5A06F0ED104
:101A000094F8463084F84E30204600F021FF636899
:101A10001B6813B10121204698470323237000233C
:101A2000A363E3632364A0E7B5F5106F32D040F6FB
:101A300002439D4252D0B5F5006F80D104F14F03AF
:101A4000A363012324E004F14C03A3630223E363B3
:101A500025648AE794F84630012B7FF470AFB4F820
:101A60004C3043F00203B6E794F84920616894F8DB
:101A700048304D6894F8471043EA0223204694F812
:101A80004620A84700283FF45AAF4368A363036881
:101A9000E363A4E72378042B10D1202383F3118878
:101AA0002046FFF7BBFE86F31188636884F84F6019
:101AB0001B68032121700BB12046984794F84630EB
:101AC000002BACD084F84F300423237063681B686C
:101AD000002BA4D0022120469847A0E7374BA363F0
:101AE0000223E36300239DE794F8481011F0800F70
:101AF000204601F00F010ED000F05EFF012806D055
:101B000002287FF41CAF2E4BA363E06367E72D4BE5
:101B1000A363E56363E700F041FFEFE794F8463025
:101B2000002B7FF40CAF94F8483013F00F013FF412
:101B300076AF1A06204602D501F0B8F96FE701F03A
:101B4000ABF96CE794F84630002B7FF4F8AE94F8CC
:101B5000483013F00F013FF462AF1B06204602D558
:101B600001F090F95BE701F083F958E7142284F85B
:101B7000342083F311882B462A4629462046FFF756
:101B80005BFE85F3118870BD5DB1152284F83420A9
:101B900083F311880021E36BA26B2046FFF74CFE14
:101BA00003E70B2284F8342083F311882B462A465E
:101BB00029462046FFF752FEE3E700BFA0390008A0
:101BC000983900089C39000838B590F8343004463C
:101BD000152B29D8DFE803F03E28282828283E289E
:101BE000280B293928282828282828283E3E90F81C
:101BF0004B1090F84A20C36B42EA01229A4214D952
:101C0000C268128AB3FBF2F502FB15356DB92023C9
:101C100083F311882B462A462946FFF71FFE85F3DA
:101C200011880A2384F8343038BD142384F8343002
:101C3000202383F3118800231A4619462046FFF714
:101C4000FBFD002383F3118838BD036C03B1984773
:101C50000023E7E7002101F015F90021204601F0FB
:101C600007F963681B6813B10621204698470623CD
:101C7000D8E7000090F83420152A38B5044622D859
:101C80000123934040F6416213421DD113F48015A5
:101C90000FD19B0217D50B2380F83430202383F318
:101CA00011882B462A462946FFF7D8FD85F311886F
:101CB00038BDC3689B695B682BB9036C03B1984757
:101CC000002384F8343038BD002101F0DBF8002116
:101CD000204601F0CDF863681B6813B10621204649
:101CE00098470623EDE70000024B00221B605B6073
:101CF0009A607047042E0020002303748268054B0D
:101D00001B6899689142FBD25A6803604260106078
:101D100058607047042E002008B5202383F31188F3
:101D2000037C032B05D0042B0DD02BB983F3118832
:101D300008BD436900221A604FF0FF334361FFF78B
:101D4000DBFF0023F2E790E80C001A6002685360A2
:101D5000F2E70000002303748268054B1B68996852
:101D60009142FBD85A680360426010605860704727
:101D7000042E0020054B19690874186802681A605F
:101D80005360186101230374FEF7BEBA042E0020CD
:101D900030B54B1C87B005460A4C10D023690A4A5F
:101DA00001A800F0D3F82846FFF7E4FF049B13B125
:101DB00001A800F007F92369586907B030BDFFF7A3
:101DC000D9FFF8E7042E0020191D000838B50C4D86
:101DD00041612B6981689A689142044603D8BDE845
:101DE0003840FFF789BF1846FFF786FF01232C61B3
:101DF000014623742046BDE83840FEF785BA00BF8F
:101E0000042E0020044B1A681B6990689B68984256
:101E100094BF002001207047042E002010B5084C0C
:101E2000236820691A6822605460012223611A74B1
:101E3000FFF790FF01462069BDE81040FEF764BA45
:101E4000042E002082600222027400224274704735
:101E50008368A3F17C0243F80C2C026943F83C2C04
:101E6000426943F8382C074A43F81C2CC26843F8EF
:101E7000102C022203F8082C002203F8072CA3F1EF
:101E8000180070472103000810B5202383F3118840
:101E9000FFF7DEFF00210446FFF798FF002383F3DE
:101EA0001188204610BD0000024B1B6958610F20AD
:101EB000FFF760BF042E0020202383F31188FFF773
:101EC000F3BF000008B50146202383F311880820E2
:101ED000FFF75EFF002383F3118808BD49B1064B6D
:101EE00042681B6918605A60136043600420FFF762
:101EF0004FBF4FF0FF307047042E00200368984218
:101F000006D01A680260506059611846FFF7F4BEA7
:101F10007047000038B504460D462068844200D161
:101F200038BD036823605C604561FFF7E5FEF4E7B8
:101F3000054B03F114025A619A614FF0FF32DA61E6
:101F400000221A62704700BF042E0020F8B503611A
:101F50001A4BC2605C6A1A4B1A46022952F8145F87
:101F600038BF0221954206461F460AD15861986142
:101F70001C620560456081600819BDE8F84001F009
:101F80006DB9186AAB68241A0C1902D3E41A2D68CB
:101F900004E09C4202D2204401F070F9AB689C42FC
:101FA000F4D86B68736035601E606E60B460A968B9
:101FB0004FF0FF33091BA960FB61F8BD000C004026
:101FC000042E002010B41A4C234653F8141F8142EB
:101FD00010D0416802680A60026851609A424FF06E
:101FE0000001C16003D0936881680B4493605DF881
:101FF000044B70470A68626100209A425360C860CF
:1020000003D15DF8044B01F033B993688868034449
:102010009360084A206A526A121A9342E7D9991AC1
:10202000012998BF931C18445DF8044B01F026B9B0
:10203000042E0020000C004000207047FEE7000046
:10204000704700004FF0FF3070470000022906D0B3
:10205000032906D00129064818BF0020704705480B
:102060007047032A9ABF044800EBC2000020704763
:10207000903A0008443A00080824002070B504464D
:1020800008460D46FEF77CFEC6B2204601340378B2
:102090000BB9184670BD32462946FEF759FE002896
:1020A000F3D1012070BD00002DE9F04F80469BB0B8
:1020B00008460C461546FEF763FE3849C6B2204670
:1020C000FFF7DCFF08B1033EF6B235492046FFF7C3
:1020D000D5FF08B11036F6B2632E01AF0CD8DFF889
:1020E000CC90DFF8CCB03E4694F800A0BAF1000FD7
:1020F0001CD186F800A003E02146384601F0DCFB45
:102100003846FEF73DFEC0B2431C5B0088E828005D
:102110002B7003236B70002302351946DAB290420C
:1021200005F1020533D81BB0BDE8F08FBAF1250FD9
:1021300028D1072219492046FEF70AFE28B9DBF804
:10214000003046F8043B0734CEE708221449204605
:10215000FEF7FEFDB0B91349B31C11F8012F1009A9
:1021600002F00F0210F8090012F8092003F8012C00
:102170000D4A03F8020C914203F10203EDD1183627
:102180000834B1E786F800A001340136ACE7FA5C08
:1021900005F8022C05F8011C0133BFE7F4390008EB
:1021A000FC3900080F7AFF1F1B7AFF1F0A3A00084C
:1021B000053A000808B5202383F311880348FFF788
:1021C00073FA002383F3118808BD00BF442E00205A
:1021D00010B50446052916D8DFE801F016150316D8
:1021E000161D202383F311880E4A0121FFF7FCFA04
:1021F00020460D4A0221FFF7F7FA0C48FFF71AFABA
:10220000002383F3118810BD202383F3118807482E
:10221000FFF7E6F9F4E7202383F311880348FFF77B
:10222000FDF9EDE7A4390008C8390008442E002064
:1022300038B50C4D0C4C0D492A4604F10800FFF747
:1022400033FF05F1CA0204F110000949FFF72CFF22
:1022500005F5CA7204F118000649BDE83840FFF7D9
:1022600023BF00BF0C330020082400201C3A0008C4
:10227000263A0008FC390008BFF34F8F024AD368A2
:10228000DB03FCD4704700BF003C024008B5094B9B
:102290001B7873B9FFF7F0FF074B1A69002ABFBF1D
:1022A000064A5A6002F188325A601A6822F4806243
:1022B0001A6008BD6A350020003C024023016745D2
:1022C00008B50B4B1B7893B9FFF7D6FF094B1A697A
:1022D00042F000421A611A6842F480521A601A6889
:1022E00022F480521A601A6842F480621A6008BDB3
:1022F0006A350020003C02400B2870B513D80B4A09
:102300000B4C137863B90B4E4FF0006144F8231067
:1023100056F8235001330C2B2944F7D101231370B5
:1023200054F8200070BD002070BD00BF9C35002017
:102330006C350020B03A0008014B53F8200070477C
:10234000B03A00080C2070470B2810B5044601D99C
:10235000002010BDFFF7D0FF064B53F8243018447F
:10236000C21A0BB9012010BD12680132F0D1043B32
:10237000F6E700BFB03A00080B2810B504461ED897
:10238000FFF77AFFFFF782FF0E49F323CB60FFF7D9
:1023900073FFC300DBB243F4007343F002030B612D
:1023A0000B6943F480330B61FFF766FFFFF7A4FF6F
:1023B000FFF786FF2046BDE81040FFF7C5BF0020AD
:1023C00010BD00BF003C02402DE9F84312F00103AC
:1023D000154643D10244B2F1016F3FD22C4B1B682A
:1023E00013F001033AD02B4CFFF750FFF323E360C7
:1023F000FFF742FF40F20127032D16D8254C0F4668
:10240000401A40F20118EB1B0B44012B00EB0706AE
:10241000236926D823F001032361FFF751FF012030
:10242000BDE8F883043D0430E6E78307E6D123697D
:1024300023F44073236123693B43236151F8046B08
:102440000660BFF34F8FFFF717FF03689E42E9D086
:10245000236923F001032361FFF732FF0020BDE869
:10246000F88323F440732361236943EA080323615B
:10247000B94637F8023B3380BFF34F8FFFF7FCFEBE
:102480003688B9F80030B6B2B342BCD0E0E700BF3E
:1024900000380240003C0240084908B50B7828B1DA
:1024A00053B9FFF7F3FE01230B7008BD23B1BDE85C
:1024B00008400870FFF704BF08BD00BF6A35002060
:1024C000014B186D704700BF00280040094B1A6F80
:1024D000120407D41A6F42F400721A671A6F42F49A
:1024E00000421A67044A136843F480731360034B75
:1024F0001865704700380240007000400028004016
:10250000034B1B689B0042BF024B01221A707047AD
:10251000743802409D350020014B1878704700BF89
:102520009D350020064A536823F001035360EFF302
:102530000983683383F30988002383F31188704784
:1025400030EF00E010B5202383F31188104B5B6857
:1025500013F4006318D0F1EE103AEFF309844FF052
:10256000807344F84C3C0B4BDB6844F8083CA4F106
:10257000680383F30988FFF745FC18B1064B44F85C
:10258000503C10BD054BFAE783F3118810BD00BF26
:1025900000ED00E030EF00E03103000834030008F4
:1025A00070470000FEE70000084A094B09498B42CA
:1025B00004D3094A0021934205D3704752F8040F0F
:1025C00043F8040BF3E743F8041BF4E75C3C000812
:1025D000903800209038002090380020836D30B56E
:1025E00000229D68446D11464FF0FF3004EB42130A
:1025F00001329542C3F80019C3F81019C3F808094D
:10260000C3F8001BC3F8101BC3F8080BEED24FF041
:102610000113C4F81C3830BD890141F0200101616B
:1026200003699B06FCD4122000F0B4BE204B03EBE0
:1026300080022DE9F047D2F80CE05D6DDEF8142041
:10264000461CD2F800C005EB063605EB4018516871
:1026500061450BD3D5F83428012303FA00F022EAB0
:102660000000C5F834081846BDE8F087BEF81040F1
:10267000ACEB0103A34228BF2346D8F81849A4B203
:10268000B3EB840F10D894681F46A4F1040959F8DD
:1026900004AFC6F800A0042F01D9043FF7E71C449B
:1026A0000B4494605360D2E70020BDE8F08700BF80
:1026B000A035002010B5054C2046FFF775F84FF007
:1026C000A0436365024BA36510BD00BFA035002089
:1026D000043B00080378012B70B5054650D12A4B06
:1026E000446D98421BD1294B5A6B42F080025A63C9
:1026F0005A6D42F080025A655A6D5A6942F0800262
:102700005A615A6922F080025A610E2143205B69A6
:10271000FEF7B4FC1E4BE3601E4BC4F800380023E8
:10272000C4F8003EC02323606E6D4FF40413A3630E
:102730003369002BFCDA012333610C2000F02AFE00
:102740003369DB07FCD4122000F024FE3369002B30
:10275000FCDA0026A6602846FFF740FF6B68C4F845
:102760001068DB68C4F81468C4F81C684BB90A4BDD
:10277000A3614FF0FF336361A36843F00103A360DB
:1027800070BD064BF4E700BFA035002000380240C2
:102790004014004003002002003C30C0083C30C020
:1027A000F8B5446D054600212046FFF735FFA96DB9
:1027B00000234FF001128F68C4F834384FF00066E0
:1027C000C4F81C284FF0FF3004EB431201339F4242
:1027D000C2F80069C2F8006BC2F80809C2F8080B19
:1027E000F2D20B686A6DEB656362102313611669A0
:1027F00016F01006FBD1122000F0CCFDD4F8003802
:1028000023F4FE63C4F80038A36943F4402343F083
:102810001003A3610923C4F81038C4F814380A4B14
:10282000EB604FF0C043C4F8103B084BC4F8003BCA
:10283000C4F81069C4F80039EB6D03F1100243F4D9
:102840008013EA65A362F8BDE03A000840800010FA
:10285000426D90F84E10D2F8003823F4FE6343EA3C
:102860000113C2F8003870472DE9F0410EB200EBB9
:1028700086080D46D8F80C100F6807F00303022BEA
:1028800050D0032B50D03D4A3D4F012B18BF174667
:10289000446D4FEA451E04EB0E030022C3F8102BD3
:1028A0008A6905F1100C002A40D04A8A05F15803C4
:1028B0005B013A43E2500123D4F81C2803FA0CF3DD
:1028C0001343A6444A69C4F81C380023CEF81039D3
:1028D00005F13F03002A39D00A8A898B9208012921
:1028E00088BF4A43C16D04EB8303561841EA024294
:1028F000C66529465A602046FFF78EFED8F80C3090
:102900001B8A43EA85531F4305F148035B01E750E7
:102910000123D4F81C2803FA05F51543C4F81C5804
:10292000BDE8F081174FB3E7174FB1E704EB46134B
:10293000D3F8002B22F40042C3F8002BD4F81C2853
:10294000012303FA0CF322EA0303BAE704EB83033F
:102950000E4A5A6004EB461629462046FFF75CFEF5
:10296000D6F8003923F40043C6F80039D4F81C38EF
:10297000012202FA05F523EA0505CFE700800010E1
:10298000008004100080081000800C100004000279
:10299000826D1268C265FFF721BE00005831436D99
:1029A00049015B5813F4004004D013F4001F14BF16
:1029B00001200220704700004831436D49015B58F7
:1029C00013F4004004D013F4001F14BF01200220B0
:1029D0007047000000EB8101CB68196A0B68136037
:1029E0004B6853607047000000EB810330B5DD6831
:1029F000AA691368D36019B9402B84BF40231360C0
:102A00006B8A1468426D1C44013CB4FBF3F46343CD
:102A1000033323F0030302EB411043EAC44343F0C2
:102A2000C043C0F8103B2B6803F00303012B09B22D
:102A30000ED1D2F8083802EB411013F4807FD0F8A1
:102A4000003B14BF43F0805343F00053C0F8003BF9
:102A500002EB4112D2F8003B43F00443C2F8003BC2
:102A600030BD00002DE9F041244D6E6D06EB4013A2
:102A70000446D3F8087BC3F8087B38070AD5D6F894
:102A80001438190706D505EB84032146DB68284670
:102A90005B689847FA072FD5D6F81438DB072BD593
:102AA00005EB8403D968CCB98B69488A5E68B6FBAC
:102AB000F0F200FB12628AB91868DA6890420DD20F
:102AC000121A83E81400202383F311880B4821464F
:102AD000FFF78AFF84F31188BDE8F081012303FA30
:102AE00004F26B8923EA02036B81CB6823B1214690
:102AF0000248BDE8F0411847BDE8F081A03500204C
:102B000000EB810370B5DD68436D6C692668E66093
:102B10004A0156BB1A444FF40020C2F810092A6833
:102B200002F00302012A0AB20ED1D3F8080803EB1F
:102B3000421410F4807FD4F8000914BF40F0805094
:102B400040F00050C4F8000903EB4212D2F800092B
:102B500040F00440C2F80009D3F83408012202FA18
:102B600001F10143C3F8341870BD19B9402E84BF78
:102B70004020206020682E8A841940F00050013CDB
:102B80001A44B4FBF6F440EAC440C6E7F8B504467C
:102B90001E48456D05EB4413D3F80869C3F808696E
:102BA000F10717D5D5F81038DA0713D500EB8403F1
:102BB000D9684B691F68DA68974218D2D21B002780
:102BC0001A605F60202383F311882146FFF798FF86
:102BD00087F31188330617D5D5F834280123A3408D
:102BE000134211D02046BDE8F840FFF71FBD012376
:102BF00003FA04F2038923EA020303818B68002BA2
:102C0000E8D021469847E5E7F8BD00BFA035002091
:102C100096482DE9F84F456D6E69AB691E4016F474
:102C2000805F6E61044605D0FEF72AFEBDE8F84FCE
:102C3000FFF788BC002E12DAD5F8003E8B489B07C0
:102C40001EBFD5F8003E23F00303C5F8003ED5F8BB
:102C5000043823F00103C5F80438FEF73BFE3705BE
:102C600002D58248FEF72AFEB0040CD5D5F8083804
:102C700013F0060FEB6823F470530CBF43F41053AA
:102C800043F4A053EB60310704D56368DB680BB1F4
:102C900076489847F2025AD4B3020CD5D4F854803F
:102CA000DFF8C8A100274FF00109A36D9B68F9B2B6
:102CB0008B4280F08780F70619D5616D0A6AC2F3EE
:102CC0000A1702F00F0302F4F012B2F5802F00F0A1
:102CD000A180B2F5402F0AD104EB830301F58051A6
:102CE000DB68186A00231A469F4240F08780300351
:102CF000D5F8184813D5E10302D50020FFF7B2FE3E
:102D0000A20302D50120FFF7ADFE630302D5022026
:102D1000FFF7A8FE270302D50320FFF7A3FE7503E4
:102D200084D5E00702D50020FFF730FFA10702D5C8
:102D30000120FFF72BFF620702D50220FFF726FFD5
:102D400023077FF573AF0320FFF720FF6EE7D4F86A
:102D50005480DFF818A100274FF00109A36D9B688C
:102D60005FFA87FB5B4597D308EB4B13D3F8002939
:102D700002F44022B2F5802F22D1D3F80029002A94
:102D80001EDAD3F8002942F09042C3F80029D3F8A4
:102D90000029002AFBDB5946606DFFF73DFC2289C4
:102DA00009FA0BF322EA0303238104EB8B03DB68AC
:102DB0009B6813B15946504698475846FFF736FC72
:102DC0000137CBE708EB4112D2F8003B03F4402374
:102DD000B3F5802F10D1D2F8003B002B0CDA6289BA
:102DE00009FA01F322EA0303638104EB8103DB6840
:102DF000DB680BB150469847013756E79C0708BF80
:102E00000A68072B98BF027003F101039CBF120AE6
:102E1000013069E7023304EB830201F58051526807
:102E200090690268D0F808C04068A2EB000E00224A
:102E3000104697420AD104EB830463689B699A6841
:102E40003A449A605A6817445F6050E712F0030FE3
:102E500008BF0868964588BF8CF8000002F101029F
:102E600084BF000A0CF1010CE3E700BFA03500208D
:102E7000436D03EB4111D1F8003B43F40013C1F85B
:102E8000003B7047436D03EB4111D1F8003943F427
:102E90000013C1F800397047436D03EB4111D1F8BD
:102EA000003B23F40013C1F8003B7047436D03EB74
:102EB0004111D1F8003923F40013C1F800397047EB
:102EC00030B5039C0172043304FB0325C361049BEA
:102ED00003630021059B00604060C16042610261A4
:102EE0008561046242628162C162436330BD000059
:102EF0000022416A41610161C2608262C2626FF078
:102F00000101FFF707B8000003694269934203D14A
:102F1000C2680AB100207047181D70470369196024
:102F2000C2680132C260C26913448269036193427C
:102F300024BF436A03610021FEF7E0BF38B50446B1
:102F40000D46E3683BB16269131D1268A362134426
:102F5000E362002038BD237A33B929462046FEF7C4
:102F6000BDFF0028EDDA38BD6FF00100FBE700007F
:102F7000C368C269013BC36043691344826943610A
:102F8000934224BF436A436100238362036B03B10E
:102F90001847704770B52023044683F31188866A6A
:102FA0003EB9FFF7CBFF054618B186F311882846D6
:102FB00070BDA36AE26A13F8015BA362934202D375
:102FC0002046FFF7D5FF002383F31188EFE70000C9
:102FD0002DE9F84F04460E4690469946202787F380
:102FE00011880025AA46D4F828B0BBF1000F09D1FA
:102FF00049462046FFF7A2FF20B18BF311882846EF
:10300000BDE8F88FA16AE36AA8EB050B5B1A9B4544
:1030100028BF9B46BBF1400F1BD9334601F140024C
:1030200051F8040B43F8040B9142F9D1A36A4033E1
:103030004036A3624035A26AE36A9A4202D3204630
:10304000FFF796FF8AF311884545D8D287F3118898
:10305000C9E730465A46FDF771FEA36A5B445E44F9
:10306000A3625D44E7E7000010B5029C01720433DF
:1030700003FB0421C36100238362C362039B0363D8
:10308000049B00604060C46042610261816104622F
:103090004262436310BD0000026AC260426A42613C
:1030A000026100228262C2626FF00101FEF732BF4C
:1030B000436902699A4203D1C2680AB1002070478D
:1030C000184650F8043B0B6070470000C368C269A3
:1030D0000133C3604369134482694361934224BF4F
:1030E000436A43610021FEF709BF000038B504467A
:1030F0000D46E3683BB123691A1DA262E2691344DD
:10310000E362002038BD237A33B929462046FEF712
:10311000E5FE0028EDDA38BD6FF00100FBE70000A6
:1031200003691960C268013AC260C26913448269C6
:103130000361934224BF436A036100238362036BEC
:1031400003B118477047000070B5202304460E46AF
:1031500083F31188856A35B91146FFF7C7FF10B1AF
:1031600085F3118870BDA36A1E70A36AE26A0133F9
:103170009342A36204D3E16920460439FFF7D0FFEC
:10318000002080F3118870BD2DE9F84F04460D46EC
:1031900091469A464FF0200888F311880026B346DE
:1031A000A76A4FB951462046FFF7A0FF20B187F329
:1031B00011883046BDE8F88FA06AE76AA9EB0603DC
:1031C0003F1A9F4228BF1F46402F1BD905F14003DD
:1031D00055F8042B40F8042B9D42F9D1A36A4033E3
:1031E000A3624036A26AE36A9A4204D3E1692046A8
:1031F0000439FFF795FF8BF311884E45D9D288F338
:103200001188CDE729463A46FDF798FDA36A3B446D
:103210003D44A3623E44E5E7026943699A4203D113
:10322000C3681BB9184670470023FBE7836A002B6D
:10323000F8D0043B9B1AF5D01360C368013BC36010
:10324000C3691A44836902619A4224BF436A0361D5
:10325000002383620123E5E700F034B9034B002229
:1032600058631A610222DA60704700BF000C004008
:10327000014B0022DA607047000C0040014B58639C
:10328000704700BF000C0040FEE7000010B5174C6F
:10329000FEF72AFDFEF74CFE802215492046FEF778
:1032A000D1FD012344F8180C0374124B124AD9685B
:1032B00021F4E0610904090C0A431049DA60CA6884
:1032C00042F08072CA600E490A6842F001020A6048
:1032D0001022DA77202283F82220002383F311883A
:1032E00062B60848BDE81040FEF7CEBD2C2E002087
:1032F000103B000800ED00E00003FA05F0ED00E0EF
:10330000001000E0183B00082DE9F84F1F4CDFF8D3
:103310008090656904F114074FF00008D9F8243053
:10332000266AAA689E1B96421DD34FF0200AAA68FF
:10333000236AD5F80CB0134423622B68BB425F604C
:10334000A6EB02066361C5F80C8001D1FFF790FF80
:1033500088F311882869D8478AF311886569AB68B2
:103360009E42E4D2DAE76269BA420CD091682362E5
:103370008E1B9660A86802282CBF1818981CBDE800
:10338000F84FFFF77BBFBDE8F88F00BF042E002089
:10339000000C0040034B59685A68521A9042FBD8FF
:1033A000704700BF001000E04B6843608B6883608B
:1033B000CB68C3600B6943614B6903628B694362ED
:1033C0000B6803607047000008B5224B22481A6959
:1033D00040F2FF110A431A611A6922F4FF7222F0C7
:1033E00001021A611A691A6B0A431A631A6D0A43B9
:1033F0001A651A4A1B6D1146FFF7D6FF184802F1ED
:103400001C01FFF7D1FF174802F13801FFF7CCFF8D
:10341000154802F15401FFF7C7FF144802F170018B
:10342000FFF7C2FF124802F18C01FFF7BDFF114800
:1034300002F1A801FFF7B8FF0F4802F1C401FFF73E
:10344000B3FF0E4802F1E001FFF7AEFFBDE8084010
:1034500000F0A4B80038024000000240383B0008E9
:103460000004024000080240000C0240001002402C
:103470000014024000180240001C024000200240DC
:1034800008B500F0FBF9FFF701FFFFF739F8BDE8D9
:103490000840FEF7CDBE000070470000084B1A69D7
:1034A000920710B508D500241C61202383F31188EE
:1034B000FFF72AFF84F31188BDE81040FFF742B8F8
:1034C000000C0040104B1A6C42F008021A641A6E8D
:1034D00042F008021A660D4A1B6E936843F0080317
:1034E00093600B4B53229A624FF0FF32DA62002254
:1034F0009A615A63DA605A6001225A6108211A609F
:103500003220FDF7BBBD00BF00380240002004E0C0
:10351000000C00401F4B1A696FEAC2526FEAD25288
:103520001A611A69C2F308021A614FF0FF301A6972
:103530005A69586100215A6959615A691A6A62F0D8
:1035400080521A621A6A02F080521A621A6A5A6A21
:1035500058625A6A59625A6A1A6C42F080521A6466
:103560001A6E42F080521A661A6E0B4A106840F4C6
:1035700080701060186F00F44070B0F5007F1EBFBF
:103580004FF4803018671967536823F40073536051
:1035900000F054B90038024000700040304B4FF04A
:1035A00080521A642F4A4FF4404111601A6842F069
:1035B00001021A601A689207FCD59A6822F0030289
:1035C0009A60274B19469A6812F00C02FBD11868D2
:1035D00000F0F90018609A601A6842F480321A60AC
:1035E0000B689B03FCD54B6F43F001034B671C4BEF
:1035F0005A6F9007FCD51C4A5A601A6842F08072D4
:103600001A60184A53685904FCD5154B1A68920180
:10361000FCD5164A9A60164B1A68164B9A42164BFE
:103620001BD1164A1168164A914216D140F2051272
:103630001A600B4B9A6842F002029A609A6802F094
:103640000C02082AFAD15A6C42F480425A645A6E2B
:1036500042F480425A665B6E704740F20572E7E7BB
:103660000038024000700040085440070094883839
:10367000002004E011640020003C024000ED00E066
:1036800041C20F41084A08B5536911680B4003F065
:103690000103536123B1054A13680BB15068984781
:1036A000BDE80840FEF74EBF003C01401038002046
:1036B000084A08B5536911680B4003F002035361CF
:1036C00023B1054A93680BB1D0689847BDE808401C
:1036D000FEF738BF003C014010380020084A08B50A
:1036E000536911680B4003F00403536123B1054A89
:1036F00013690BB150699847BDE80840FEF722BF37
:10370000003C014010380020084A08B55369116890
:103710000B4003F00803536123B1054A93690BB1D1
:10372000D0699847BDE80840FEF70CBF003C014057
:1037300010380020084A08B5536911680B4003F09F
:103740001003536123B1054A136A0BB1506A9847BD
:10375000BDE80840FEF7F6BE003C014010380020EE
:10376000174B10B55C691A68144004F478725A61FA
:10377000A30604D5134A936A0BB1D06A9847600632
:1037800004D5104A136B0BB1506B9847210604D532
:103790000C4A936B0BB1D06B9847E20504D5094AEC
:1037A000136C0BB1506C9847A30504D5054A936C74
:1037B0000BB1D06C9847BDE81040FEF7C3BE00BF08
:1037C000003C0140103800201A4B10B55C691A68A3
:1037D000144004F47C425A61620504D5164A136D04
:1037E0000BB1506D9847230504D5134A936D0BB167
:1037F000D06D9847E00404D50F4A136E0BB1506E9C
:103800009847A10404D50C4A936E0BB1D06E98472B
:10381000620404D5084A136F0BB1506F9847230414
:1038200004D5054A936F0BB1D06F9847BDE810409F
:10383000FEF788BE003C014010380020062108B584
:103840000846FDF71BFC06210720FDF717FC0621A3
:103850000820FDF713FC06210920FDF70FFC0621C7
:103860000A20FDF70BFC06211720FDF707FC0621B7
:103870002820BDE80840FDF701BC000008B5FFF7AF
:1038800049FE00F00DF8FDF79FFDFDF78BFFFDF7FA
:103890005FFEFFF701FEBDE80840FFF7DDBC00005A
:1038A000002304491A465A50C8180833802B426036
:1038B000F9D1704710380020034611F8012B03F8A6
:1038C000012B002AF9D170471210121312110000B7
:1038D00053544D3332463F3F3F000000000000008C
:1038E000D03800083F00000013040000143900081D
:1038F0003F000000190400001E3900083F000000CE
:1039000021040000283900083F000000442E002058
:103910009C29002053544D333246343078005354A0
:103920004D3332463432780053544D3332463434BA
:10393000365858000096000000000000000000000B
:1039400000000000000000000000000091130008CB
:103950007D130008B9130008A5130008B11300086F
:103960009D1300088913000875130008C51300088B
:1039700000000000C9140008B5140008F114000884
:10398000DD140008E9140008D5140008C11400086B
:10399000AD1400084D1500080000000001000000F3
:1039A000000000000200000000000000F516000802
:1039B0005D17000840004000DC320020EC3200209F
:1039C00002000000000000000300000000000000F2
:1039D000A11700080000000010000000FC320020C9
:1039E000000000000100000000000000A0350020E1
:1039F0000101020025424F41524425002553455202
:103A000049414C2500463442590030313233343577
:103A100036373839414243444546000041726475A7
:103A200050696C6F740025424F415244252D424C21
:103A300000000000D12100084D2000086116000898
:103A4000B5210008430000004C3A00080902430079
:103A5000020100C032090400000102020100052435
:103A600000100105240100010424020205240600BF
:103A700001070582030800FF09040100020A000093
:103A80000007050102400000070581024000000018
:103A900012000000983A00081201100102000040D4
:103AA00083044057000201020301000004030904DB
:103AB0000040000000400000004000000040000006
:103AC00000000100000002000000020000000200EF
:103AD00000000200000002000000020000000200DE
:103AE00000000000E9180008C91B0008751C000848
:103AF0004000400000360020003600200100000099
:103B0000103600208000000040010000030000008B
:103B10006D61696E00000000303B0008183600201F
:103B20001038002001000000893200080000000069
:103B300069646C65000000000000802A000000003D
:103B4000AAAAAAAA00000000FFFF000000000000CF
:103B500000A00A000000000000000000AAAAAAAA13
:103B600000000000FFFF0000000000000000000057
:103B70000000000000000000AAAAAAAA000000009D
:103B8000FFFF00000000000000000000002800000F
:103B900000000000AAAAAAAA00140000FFFF00006B
:103BA000000070070000000050000000000000004E
:103BB000AAAAAAAA00000000FFFF0000000000005F
:103BC000000000000000000000000000AAAAAAAA4D
:103BD00000000000FFFF00000000000000000000E7
:103BE0000000000000000000AAAAAAAA000000002D
:103BF000FFFF0000000000000000000000000000C7
:103C0000000000000A0000000000000003000000A7
:103C100000000000000000000000000000000000A4
:103C20000000000000000000000000000000000094
:103C30000000000000000000FF00960000000008E7
:103C400004000000AC3A0008000000000000000082
:103C50000000000000000000000000000000000064
:00000001FF
